:100000000F28FF3FFF3FFF3F0B110900F6000030B4
:100010008A000F30760703188A0A76088207203094
:1000200083120313BB000430BC000230BD00D601B4
:1000300083120313D7010930D8000230D9000130F0
:10004000DA000230DB000830DC000130DD00043073
:100050008600F03083168500F23086004030810043
:100060008B01C6260730831203139F0019308316B5
:100070009900243098009030831298008C01B701C9
:100080000130B600B901B8013030CA003C27B701D1
:100090000230B600B901B8014030CA003C27FA303E
:1000A000B4007927FA30B4007927FA30B400792700
:1000B000032783120313B7010230B600B901B80158
:1000C000CA013C27D224D224831203130608F0006D
:1000D000F00CF00CF00C700C0F39F0007008063CBE
:1000E000031D7C2883120313A001A101A201A30117
:1000F0008F30A400B7240F2A7008073C031DDF28A7
:100100000130831203135A02031DB628053057022B
:10011000013003180301F1005708073C01300318B0
:1001200003017104003C0319AF285708093C013052
:1001300003190301F10057080B3C013003190301B7
:100140007105003C0319AF285708A000A101A201C6
:10015000A3010730A400B72483120313CC00D70AED
:100160000D305702031D0F2AD7010F2A02308312C8
:1001700003135A02031DC52806305D02031DC32860
:100180000130DD00DE28DD0ADE2803308312031390
:100190005A02031DDE28A001A101A201A3015C08EF
:1001A000A400B72483120313CC0008305C02031DA3
:1001B000DC288830DC00DE280830DC000F2A7008DC
:1001C0000B3C031D82290130831203135A02031DC5
:1001D0005C29CB019727593083120313CB00972753
:1001E00083120313CB01972783120313CB019727A5
:1001F000BB3083120313CB009727A627FE00A62748
:10020000FF000130831203135302031D2329F10160
:100210007E08103E0318F10AFE00F100F10CF10C0B
:10022000F10C710C0F390E3C031D3C297E08F100C6
:10023000710EF039F039F100F10CF10CF10C710C88
:100240000F39FE003C29F1017E08013E0318F10A36
:10025000FE00F100710EF039F039E03C031D3C293D
:100260007E08F100F10CF10CF10C710C0F39F1006A
:10027000710EF039F039FE0083120313CB0197277A
:10028000593083120313CB0097277E088312031380
:10029000CB0097277F0883120313CB009727BC302E
:1002A00083120313CB009727A62783120313CC00D6
:1002B0000A30B40079270F2A02305A02031D6B2935
:1002C000C2015D08C30012250130A400B7248312C7
:1002D0000313CC00812903305A02031D8129A00198
:1002E000A101A201A3015B08A400B7248312031398
:1002F000CC00CC08031D7F298230DB00812902302D
:10030000DB000F2A70080D3C031DC7290130831242
:1003100003135A02031D9729A001A101A201A30101
:100320008130A400B72483120313CC000F2A0230BB
:100330005A02031DA7290130C2005D08C30012251F
:100340000130A400B72483120313CC00C629033064
:100350005A02031DC6295808A000A101A201A30149
:100360000930A400B72483120313CC0009305802CB
:10037000031DBD294930D800C62949305802031D44
:10038000C4298930D800C6290930D8000F2A70083E
:100390000E3C031D0F2A0430831203135902031D60
:1003A000D3290130D9003230B40079275908F1003F
:1003B0007108013C031DE82983120313B7010230C1
:1003C000B600B901B801CA013C270130DA000B2A96
:1003D0007108023C031DF92983120313B70102308F
:1003E000B600B901B8011030CA003C270230DA006B
:1003F0000B2A7108033C031D0B2A83120313B70158
:100400000230B600B901B8012030CA003C270330E1
:10041000DA000B2A0B2A83120313D90A0F2AD224DB
:10042000CB019727553083120313CB0097278312F4
:100430000313CB01972783120313CB019727BB30FC
:1004400083120313CB009727A627FE00A627FF00E1
:100450007E088039003C0319692A7E08F000700884
:10046000813C031D3A2A423083120313CF0001302E
:10047000D300742A7008803C031D442A4130831243
:100480000313CF00D301742A7008903C031D492A3E
:100490004D2A7008913C031D502A4830CF00742A21
:1004A0007008843C031D552A592A7008853C031D99
:1004B0005C2A5130CF00742A7008863C031D612AE3
:1004C000652A7008873C031D682A7430CF00742A9F
:1004D000742A4D3083120313CF007E082039003C6C
:1004E0000319742A5430CF000130BF00C0014F08F7
:1004F000C1000425F0013030F100831203132508F8
:10050000F200F20CF20CF20C720C0F3971070318A6
:10051000F00AAA00303C031D8F2A2030AA00F00107
:100520003030F1002508F200720EF039F039F20097
:10053000F20CF20CF20C720C0F3971070318F00A6E
:10054000AB002A08203C0130031D0301F0002B08FA
:10055000303C0130031D03017005003C0319B22A31
:100560002030AB00F0013030F1002608F200F20C30
:10057000F20CF20C720C0F3971070318F00AAC0080
:100580002E30AD00F0013030F1002608F200720E7E
:10059000F039F039F200F20CF20CF20C720C0F3957
:1005A00071070318F00AAE00F0013030F10027089F
:1005B000F200F20CF20CF20C720C0F3971070318F6
:1005C000F00AAF00F0013030F1002708F200720E9F
:1005D000F039F039F200F20CF20CF20C720C0F3917
:1005E00071070318F00AB0002E30B100F00130306E
:1005F000F1002808F200F20CF20CF20C720C0F3928
:1006000071070318F00AB200F0013030F100280839
:10061000F200720EF039F039F200F20CF20CF20C2A
:10062000720C0F3971070318F00AB3005608093C21
:10063000031C2F2B0130BF00F001023056070318B6
:10064000F00AC00056082A3E840083130008831273
:100650000313C100042583120313D60A162BD601F7
:100660005608023C031C582B0130BF00F0010D302E
:1006700056070318F00AC0002908F7000330F800F5
:10068000C227F0007808583EF1000318F00A7108FC
:10069000831203135607F1000318F00A7108BE0015
:1006A000FC248312C100042583120313D60A302BC5
:1006B000D60101305302031D622B0330D4003C30BD
:1006C000D500662B0130D400B630D5005408CB00DD
:1006D0009727831203135508CB0097278312031320
:1006E000CB01972783120313CB019727BB308312CB
:1006F0000313CB009727A627FE00A627FF007E083E
:10070000643C031D882B2D3083120313D000932BE0
:100710007E08A43C031D912B2B3083120313D000C1
:10072000932B2030D0000130BF000C30C0005008A7
:10073000C100042583120313CB019727793083125C
:100740000313CB00972783120313CB019727831240
:100750000313CB019727BB3083120313CB009727DA
:10076000A627FE00A627FF007E08F000700EF039D5
:10077000F039F0007008003C031DBF2BC32B70083C
:10078000403C031DC82B343083120313CE00EE2BE4
:100790007008103C031DCD2BD12B7008503C031D5D
:1007A000D62B333083120313CE00EE2B7008203C7F
:1007B000031DDB2BDF2B7008603C031DE22B323066
:1007C000CE00EE2B7008303C031DE72BEB2B70089E
:1007D000703C031DEE2B3130CE00EE2B0230BF00FB
:1007E0000530C0004E08C10004257F088039003C58
:1007F0000319082C0330831203135A02031D112C12
:100800000230BF000C30C0002A30C1000425112C7A
:10081000023083120313BF000C30C0002030C1002F
:10082000042583120313A001A101A201A301F73043
:10083000A400B72483120313CC008039031D3C2C81
:100840000230BF00C0015030C100042583120313E1
:100850004C1F322C0230BF000330C0004830C100B2
:100860000425592C023083120313BF000330C0004B
:100870004C30C1000425592C023083120313BF00F1
:10088000C0017330C100042583120313A001A1012C
:10089000A201A301E730A400B72483120313CC0004
:1008A0008039031D592C0230BF00C0015330C100F4
:1008B0000425831203134C08F000700EF039F03950
:1008C000F000F00CF00CF00C700C0F39CD00013082
:1008D0004D02031C882C01304D020130031C030122
:1008E000F0004D08093C0130031C03017005003C79
:1008F0000319832CF00130304D070318F00AD100A2
:100900002030D2008D2C3930D1002B30D2008D2CEC
:10091000203083120313D100D2000230BF00013017
:10092000C0005108C1000425023083120313BF0028
:10093000C0005208C10004250230831203135A027A
:10094000031DAD2C0230BF000F30C000F00130306D
:100950005D070318F00AC100042502308312031357
:10096000BF000630C0007C30C1000425642883121B
:1009700003132008CB009727831203132108CB0011
:100980009727831203132208CB00972783120313A0
:100990002308CB009727831203132408CB00972743
:1009A000A627080083120313CB0197278312031392
:1009B000CB01972783120313CB01972783120313CD
:1009C000CB019727033083120313CB009727A62769
:1009D00083120313A500A62783120313A600A627DC
:1009E00083120313A700A62783120313A800A627C8
:1009F00083120313A9000800831203133E08831611
:100A00009B001C141A080800831203133F08C80037
:100A10004008C9000F278312031306144108C700BA
:100A2000EC260800303083120313E0003930E10077
:100A30004208003C0319212D6108DE006008DF0038
:100A4000252D6008DE006108DF004308063C031C1A
:100A5000592E33085E020130031D0301F1000230FC
:100A600043020130031C0301F2004308063C01303D
:100A7000031C030172057104003C03194E2E013062
:100A80004302031D452D5F08B30032085E020130AA
:100A9000031D0301F100033043020130031C030175
:100AA000F2004308063C0130031C03017205710487
:100AB000003C0319432E4308013C0130031D030190
:100AC000F1004308023C0130031D03017104003CA6
:100AD00003196C2D5F08B20030085E020130031D5F
:100AE0000301F100043043020130031C0301F20052
:100AF0004308063C0130031C030172057104003CED
:100B00000319312E013043020130031C0301F100AF
:100B10004308033C0130031C03017105003C031929
:100B2000932D5F08B0002F085E020130031D030102
:100B3000F100053043020130031C0301F2004308B9
:100B4000063C0130031C030172057104003C0319CB
:100B5000262E013043020130031C0301F10043083B
:100B6000043C0130031C03017105003C0319BA2D3C
:100B70005F08AF002E085E020130031D0301F10083
:100B80004308063C0130031D03017104003C0319B6
:100B90001B2E013043020130031C0301F100430806
:100BA000053C0130031C03017105003C0319DA2DDB
:100BB0005F08AE002C085E02031D102E01304302B8
:100BC0000130031C0301F1004308063C0130031C03
:100BD00003017105003C0319EF2D5F08AC002B08E1
:100BE0005E02031D052E5F08AB002A085E02031D8E
:100BF000FC2D5F08AA00592E2A08C4004208C5002F
:100C00000130C600B426AA00592E831203132B0804
:100C1000C4004208C5000130C600B426AB00592EFE
:100C2000831203132C08C4004208C5000130C6001B
:100C3000B426AC00592E831203132E08C4004208B8
:100C4000C5000130C600B426AE00592E831203132E
:100C50002F08C4004208C5000130C600B426AF000A
:100C6000592E831203133008C4004208C500013016
:100C7000C600B426B00003304302031D422E3030BC
:100C8000B200B300592E831203133208C400420885
:100C9000C5000130C600B426B200592E83120313DA
:100CA0003308C4004208C5000130C600B426B300B2
:100CB000592EF101831203132A08F200720EF03943
:100CC000F039F2002B08F300730EF039F039F3001D
:100CD000F30CF30CF30C730C0F3972070318F10AC1
:100CE000A000F1012C08F200720EF039F039F20088
:100CF0002E08F300730EF039F039F300F30CF30C07
:100D0000F30C730C0F3972070318F10AA100F101FB
:100D10002F08F200720EF039F039F2003008F300BB
:100D2000730EF039F039F300F30CF30CF30C730C81
:100D30000F3972070318F10AA200F1013208F2001C
:100D4000720EF039F039F2003308F300730EF03907
:100D5000F039F300F30CF30CF30C730C0F3972073A
:100D60000318F10AA3000800831203134508003C8E
:100D70000319C12EF101440846070318F10AC40003
:100D8000C42E46084402C40044080800831203131A
:100D9000861106100530B400792703308500FE2641
:100DA0000530B400792702308500FE260530B400F6
:100DB00079272830C700EC26083083120313C700B8
:100DC000EC260C3083120313C700EC260630831286
:100DD0000313C700EC260800831203134708F3002F
:100DE000F30CF30CF30C730C0F398500FE26470847
:100DF0008500FE262830BA008A27080083120313D4
:100E00008615861108008312031306100130C700EF
:100E1000EC26023083120313B400792708008312F2
:100E2000031306104808F2007208013C031D222F2C
:100E3000F30180308312031349070318F30AC70034
:100E4000EC26362F7208023C031D362FF30140308A
:100E50008312031349070318F30AF40073080038D8
:100E6000F30074088038C700EC26362F0230831256
:100E70000313B4007927080083120313DE01DF0196
:100E80005F08003C0030031C4D2F0130031D4D2F27
:100E90005E080F3C0130031C0301003C0319782F4E
:100EA0003708F2003608C8003908F2005F08F20778
:100EB00038085E070318F20AC9000F2783120313CC
:100EC00006140030F2005F08F2074A085E070318B4
:100ED000F20ABE00FC24013CF2007209013E8312BA
:100EE000C700EC2683120313DE0A0319DF0A402F22
:100EF00008008E3083120313B500000000000000CC
:100F0000000000000000B50B7F2F0000B40B792F0C
:100F10000000080083120313BA0CBA0C3F30BA0564
:100F20000330BA020000BA0B922F000008008312AF
:100F300003134B0899008316831203130108031946
:100F4000A42F831618089C2F831208008312031302
:100F50000C083B05FF39003C0319A62F18083C0577
:100F6000FF39F10018083D05FF397104003C0319F1
:100F7000BE2F1812000018161A08E2001A080800FE
:100F8000A62F08000930F9007708F7010310F70CC5
:100F9000F80C0318F707F90BC72F77080800FF3F75
:100FA000FF3FFF3FFF3FFF3FFF3FFF3FFF3FFF3F51
:100FB000FF3FFF3FFF3FFF3FFF3FFF3FFF3FFF3F41
:100FC000FF3FFF3FFF3FFF3FFF3FFF3FFF3FFF3F31
:100FD000FF3FFF3FFF3FFF3FFF3FFF3FFF3FFF3F21
:100FE000FF3FFF3FFF3FFF3FFF3FFF3FFF3FFF3F11
:100FF000FF3FFF3FFF3FFF3FFF3FFF3FFF3FFF3F01
:084000000F000F000F000F007C
:02400E00503F21
:104200002100210021002100210021002100570070
:10421000670021004300650021004E006500210079
:104220002100210021002100210021002100560051
:104230007100210045007800210054007500210024
:104240002100210021002100210021002100530034
:10425000710021005400710021005100550021001F
:10426000470055002E00390032003800210053006D
:1042700066006E007000750066004E0062006F0000
:104280004A00580033004D004700450021007300EC
:1042900032002F003300210033003100310035009F
:1042A00020002000720031002E0032002E0031006C
:1042B0004C005300420055005300420020004300D0
:1042C0005700430057005200200041004D000000FD
:1042D00000000000570046004D00000000000000F4
:1042E000200046004D00000000000000440049008E
:1042F000470000000000000050004B005400000088
:00000001FF
